S0220000687474703A2F2F737265636F72642E736F75726365666F7267652E6E65742F1D
S12300000C9438000C94D71D0C94AB170C945F000C945F000C945F000C945F000C945F0013
S12300200C945F000C943F200C945F000C9416240C945F000C944D180C9427180C94041747
S12300400C9416250C945F000C9495240C945F000C94B1250C9479250C945F000C945F00B8
S12300600C945F000C945F000C945F000C945F0011241FBECFEFD0E1DEBFCDBF14BEA895C7
S123008088E10FB6F89480936000109260000FBE15E0A0E0B1E0ECEDFEE402C005900D92A9
S12300A0A632B107D9F716E0A6E2B5E001C01D92A63EB107E1F70E94BA100C946D270C94A5
S12300C0000020E030E0D901AC54BF4F0E944F27802DF901EE5BFE4F80832F5F3F4F203A56
S12300E0310589F720E030E0D901A857BE4F0E944F27802DF901E55CFE4F80832F5F3F4FE4
S12301002530310589F712BC11BC089520E030E0F901EE5BFE4F8081D901AC54BF4F082ED9
S12301200E945C272F5F3F4F203A310589F712BC11BC0895349B11C020E030E0D9015096C2
S12301400E944F27802DF901EE51FE4F80832F5F3F4F203A310591F0F1CF20E030E0D90176
S1230160A859BD4F0E944F27802DF901EE51FE4F80832F5F3F4F203A310589F712BC11BC59
S12301800895349B11C020E030E0F901EE51FE4F8081D9015096082E0E945C272F5F3F4F50
S12301A0203A310591F0F1CF20E030E0F901EE51FE4F8081D901A859BD4F082E0E945C2791
S12301C02F5F3F4F203A310589F712BC11BC089520E931E0D9010E944F27802D2055314018
S12301E0F901EE57FD4F80832F5A3E4F81E0203F380781F712BC11BC089520E430E0F9019A
S1230200EE57FD4F8081D901A05BBE4F082E0E945C272F5F3F4F203A310589F712BC11BC44
S12302200895A2E0B0E00E944F27802D90E090931D0180931C0120911C0130911D01A3E035
S1230240B0E00E944F27802D90E0982F8827820F931F90931D0180931C01ADEEB3E00E94DB
S12302604F27802D90E090932101809320012091200130912101AEEEB3E00E944F27802DC5
S123028090E0982F8827820F931F909321018093200180911C0190911D0190931F018093F5
S12302A01E01A4E0B0E00E944F27802D90E090932301809322012091220130912301A5E017
S12302C0B0E00E944F27802D90E0982F8827820F931F9093230180932201A6E0B0E00E9467
S12302E04F27802D90E090930101809300012091000130910101A7E0B0E00E944F27802DDD
S123030090E0982F8827820F931F9093010180930001A1E0B0E00E944F27802D8093260563
S1230320A8E0B0E00E944F27802D80931301A9E5B1E00E944F27802D80932C01A2E0B4E07B
S12303400E944F27902D892F8150843078F080912C01843039F481E08093180183E68093F7
S1230360E60506C082E08093180102C090931801A9E0B0E00E944F27802D80931201AEE0AA
S1230380B0E00E944F27802D80932501ABE0B0E00E944F27802D80931901ACE0B0E00E9400
S12303A04F27802D80931A01AFE6B1E00E944F27802D80931B01A2EFB1E00E944F27802DE7
S12303C080939A0580919A05882319F081E080939A05ADE0B0E00E944F27802D26E0829FE7
S12303E0C00111249093150180931401A1E7B1E00E944F27802D80930A06A0E7B1E00E94E7
S12304004F27802D809308068AE08093390681E080933706AFE8B1E00E944F27802D809327
S12304202D0180912D0181FF05C080912D01827F80932D0180912D0185FF05C080912D01BE
S12304408F7280932D01A4EFB1E00E944F27802D90E02CE231E0AC01429FC001439F900D10
S1230460529F900D11249093E1058093E005A5EFB1E00E944F27802D8093DD05A6EFB1E0AF
S12304800E944F27802D8093DB05A7EFB1E00E944F27802D8093DA05A8EFB1E00E944F2782
S12304A0802D90E09093D9058093D8052091D8053091D905A9EFB1E00E944F27802D90E09F
S12304C0982F8827820F931F9093D9058093D805ABEFB1E00E944F27802D90E090932F01BB
S12304E080932E0120912E0130912F01ACEFB1E00E944F27802D90E0982F8827820F931FCB
S123050090932F0180932E01ADEFB1E00E944F27802D90E090933101809330012091300165
S123052030913101AEEFB1E00E944F27802D90E0982F8827820F931F90933101809330010F
S1230540AFEFB1E00E944F27802D90E09093B5048093B4042091B4043091B504A0E0B2E097
S12305600E944F27802D90E0982F8827820F931F9093B5048093B40420E030E0D901A25AFC
S1230580BE4F0E944F27802DF901EE5DFC4F8083D901AE58BE4F0E944F27802DF901E9510C
S12305A0FA4F8083D901A458BE4F0E944F27802D808B2F5F3F4F2A30310501F7A7E0B2E07B
S12305C00E944F27802D80933601A3E0B2E00E944F27802D8093370120E030E0F901EA5E91
S12305E0F94F84E6808BD901A45EBD4F0E944F27802D80832F5F3F4F2031310579F720E077
S123060030E0D901A759BE4F0E944F27802DF901E95DFE4F80832F5F3F4F2430310589F764
S123062020E030E0D901A25DBD4F0E944F27802DF901E750FB4F80832F5F3F4F20313105DB
S123064089F7ADE6B1E00E944F27802D80932401A1EFB1E00E944F27802D80939905A0EFCF
S1230660B1E00E944F27802D80932B01A6E0B2E00E944F27802D8093260120E030E0D901E0
S1230680AA54BC4F0E944F27802DF901E45DFC4F80832F5F3F4F2031310589F7A7ECB3E0B6
S12306A00E944F27802D80933901A8ECB3E00E944F27802D80933A01A4EDB3E00E944F27AE
S12306C0802D8093A005A5EDB3E00E944F27802D8093A105A6EDB3E00E944F27802D809310
S12306E0A205A7EDB3E00E944F27802D8093A305A8EEB3E00E944F27802D90E090933301F3
S1230700809332012091320130913301A9EEB3E00E944F27802D90E0982F8827820F931F9E
S12307209093330180933201AAEEB3E00E944F27802D80939C0512BC11BC089580911C010E
S123074090911D01A2E0B0E0082E0E945C2780911C0190911D01892F9927A3E0B0E0082EBB
S12307600E945C278091220190912301A4E0B0E0082E0E945C278091220190912301892F37
S12307809927A5E0B0E0082E0E945C278091000190910101A6E0B0E0082E0E945C2780916E
S12307A0000190910101892F9927A7E0B0E0082E0E945C2780911301A8E0B0E0082E0E9412
S12307C05C2780911201A9E0B0E0082E0E945C2712BC11BC089580E0A1EFB1E0082E0E9469
S12307E05C278AE0A0EFB1E0082E0E945C2780919A05A2EFB1E0082E0E945C2784E0A9E56E
S1230800B1E0082E0E945C2785E0ACE0B0E0082E0E945C2782E3AFE6B1E0082E0E945C2726
S123082024E1A1E7B1E0022E0E945C2791E0A0E7B1E0092E0E945C2788ECA4EFB1E0082E8E
S12308400E945C27A5EFB1E0092E0E945C27A6EFB1E0022E0E945C278AE5A7EFB1E0082EA7
S12308600E945C2788EEA8EFB1E0082E0E945C2783E0A9EFB1E0082E0E945C2780912E012F
S123088090912F01ABEFB1E0082E0E945C2780912E0190912F01892F9927ACEFB1E0082E12
S12308A00E945C278091300190913101ADEFB1E0082E0E945C278091300190913101892FA5
S12308C09927AEEFB1E0082E0E945C278091B4049091B504AFEFB1E0082E0E945C2780918D
S12308E0B4049091B504892F9927A0E0B2E0082E0E945C278CEDA7E0B2E0082E0E945C2790
S123090086EEA3E0B2E0082E0E945C272CE132E088ECD901082E0E945C272F5F3F4F82E0A9
S12309202C323807A9F782E2AFE8B1E0082E0E945C2781E0A6E0B2E0082E0E945C2712BCED
S123094011BC0895CF92DF92EF92FF920F931F93CF93DF93C0E0D0E0A5E0B2E00E944F279E
S1230960202D30E040E050E0A3EDB3E00E944F27602D6E01CC0CDD1C8CE393E0C80ED91E0F
S1230980F601E080F18070E080E090E00E94C02600E010E0A80197010E94C02624E630E030
S12309A040E050E00E94122779018A01CA01B90124EF31E040E050E00E94C02628EC30E05E
S12309C040E050E0E20EF31E041F151FA80197010E941227CA01B9012FEF30E040E050E04C
S12309E00E94C02625E030E040E050E00E941227E2E0220F331F441F551FEA95D1F7CA01FD
S1230A00B90124E630E040E050E00E941227F601318320832196C732D10509F09DCFC0E0FA
S1230A20D0E0A9ECB3E00E944F27202D30E040E050E0A3EDB3E00E944F27602D6E01CC0C06
S1230A40DD1C8AE893E0C80ED91EF601E080F18070E080E090E00E94C02600E010E0A801FE
S1230A6097010E94C02624E630E040E050E00E94122779018A01CA01B90124EF31E040E03F
S1230A8050E00E94C02628EC30E040E050E0E20EF31E041F151FA80197010E941227CA01E7
S1230AA0B9012FEF30E040E050E00E94C02625E030E040E050E00E94122792E0220F331F3D
S1230AC0441F551F9A95D1F7CA01B90124E630E040E050E00E941227F60131832083219675
S1230AE0C732D10509F09DCFC0E0D0E0AAECB3E00E944F27202D30E040E050E0A3EDB3E05D
S1230B000E944F27602D6E01CC0CDD1C88ED93E0C80ED91EF601E080F18070E080E090E04F
S1230B200E94C02600E010E0A80197010E94C02624E630E040E050E00E94122779018A0146
S1230B40CA01B90124EF31E040E050E00E94C02628EC30E040E050E0E20EF31E041F151F44
S1230B60A80197010E941227CA01B9012FEF30E040E050E00E94C02625E030E040E050E065
S1230B800E94122702E0220F331F441F551F0A95D1F7CA01B90124E630E040E050E00E9442
S1230BA01227F601318320832196C732D10509F09DCFC0E0D0E0A4E0B2E00E944F27202DF4
S1230BC030E040E050E0A3EDB3E00E944F27602D6E01CC0CDD1C86E294E0C80ED91EF60109
S1230BE0E080F18070E080E090E00E94C02600E010E0A80197010E94C02624E630E040E0A5
S1230C0050E00E94122779018A01CA01B90124EF31E040E050E00E94C02628EC30E040E0FB
S1230C2050E0E20EF31E041F151FA80197010E941227CA01B9012FEF30E040E050E00E9467
S1230C40C02625E030E040E050E00E941227B2E0220F331F441F551FBA95D1F7CA01B901E2
S1230C6024E630E040E050E00E941227F601318320832196C732D10509F09DCFDF91CF9122
S1230C801F910F91FF90EF90DF90CF900895EAE7F0E0108210927C0080E880BF87EE808317
S1230CA011B888E790E0909329058093280584E690E0909337058093360508950F931F937F
S1230CC0CF93DF93282F30E0F901EE0FFF1FEE5FFE4F0081118143E0033F140718F0E2E3C6
S1230CE0F0E04CC053E00F3D150718F0EAE0F0E045C0C0E0D0E087E290E0A901489F900187
S1230D00499F300D589F300D1124D901AC0FBD1FAA0FBB1FA45CBC4F8D919C9111978017A8
S1230D20910730F5FE013197E20FF31FEE0FFF1FE45CFC4F20813181608171814D915C9191
S1230D40FE01EE0FFF1FEE0FFF1FEC0FFD1F3596201B310BC901880F991F880F991F641B1A
S1230D60750B820F931F0E94EB26E60FF71F06C02196C732D10549F6E8ECF0E0CF01DF917F
S1230D80CF911F910F9108950F931F93CF93DF93AC01E0E0F0E0EF01CC0FDD1FDE01AC58F3
S1230DA0BB4F8D919C91119748175907C0F56D917C913197EE0FFF1FDF01AC58BB4F8D91C4
S1230DC09C911197681B790B8D919C91C457DB4F28813981E457FB4F00811181481B590BE1
S1230DE084E690E0DC014A9FC0014B9F900D5A9F900D11240E94EB26201B310B0190F08110
S1230E00E02D629FC001639F900D729F900D112464E670E00E94EB266E0F7F1F09C0319685
S1230E20EA30F10509F0B7CF6091A0047091A104CB01DF91CF911F910F910895809128051D
S1230E4090912905282F205527FF0AC08091140190911501BC01660F771F680F791F1EC071
S1230E602F312CF0609114017091150117C04091140150911501332727FD309588E290E004
S1230E80821B930B9C01249FC001259F900D349F900D11246AE070E00E94EB26CB01089536
S1230EA00F931F93CF93DF93AC018091B7049091B8044817590718F4E0EFF0E057C080911E
S1230EC0D3049091D4048417950718F4E0E0F0E04DC0E1E0F0E0EF01CC0FDD1FDE01A9542A
S1230EE0BB4F8D919C91119748175907C0F56D917C913197EE0FFF1FDF01A954BB4F8D918A
S1230F009C911197681B790B8D919C91EB52FB4F20813181CB52DB4F08811981481B590B9B
S1230F2084E690E0DC014A9FC0014B9F900D5A9F900D11240E94EB26201B310B0190F081CE
S1230F40E02D629FC001639F900D729F900D112464E670E00E94EB26E61BF70B07C031965E
S1230F60EE30F10509F0B7CFEEEFF0E0CF01DF91CF911F910F9108958091A705882359F0EF
S1230F808CED95E090933501809334011092B3051092B2052AC08091A705882349F08CED07
S1230FA095E0909335018093340184E690E019C08091A705882349F08CED95E0909335017C
S1230FC0809334018AEF90E00CC08091A705882361F08CED95E0909335018093340184EF55
S1230FE091E09093B3058093B205F89480919505909196058A5A9A4AC1F08091950590919F
S123100096058555954589F0789480911406909115068064909315068093140684EF91E05E
S123102090933501809334010AC0789480911406909115068F7B9093150680931406F894CD
S123104080919705909198058F5F9F4F89F078948091140690911506806890931506809320
S1231060140684EF91E090933501809334010AC0789480911406909115068F77909315064C
S1231080809314068091340190913501892B91F1429A2091B2053091B3052115310511F41E
S12310A0429A15C08091B0059091B105029778F488B18695869580958170880F880F98B1ED
S12310C09B7F982B98B93093B1052093B0058091B0059091B10501979093B1058093B00527
S12310E0809134019091350101979093350180933401089542981092B3051092B20508954F
S123110080911406909115069F779093150680931406809100019091010197FD44C0809105
S1231120260580FF32C020918D0530918E0580911E0190911F018C599F4F8217930720F4ED
S123114061E070E040E832C020918D0530918E0580911E0190911F0149978217930720F4B1
S123116061E070E048E022C020918D0530918E0580911E0190911F018456904082179307EB
S123118090F461E070E044E011C020918D0530918E0580911E0190911F018217930718F4FA
S12311A060E070E802C060E070E040E02091140630911506CB019927869597958827822B4B
S12311C0932B90931506809314062091140630911506CB0180709078822B932B90931506CE
S12311E08093140620913605309137058091370190E08217930734F480913701882311F0CC
S1231200606148608091A105209138053091390590E08F5B9F4F8217930774F48091A10523
S1231220882351F0606280918D0590918E05895B9B40A0F0446012C08091A105209138053B
S12312403091390590E0C296821793073CF48091A105882319F0606251E001C050E0809100
S1231260A00520913E0530913F0590E0C296821793076CF48091A005882349F06064809102
S12312808D0590918E05855C994008F04460552321F082E38093890502C01092890570932A
S12312A0A6056093A5054093A7050895809100019091010193FF6FC0339B06C08091AC057A
S12312C08F5F8093AC0502C01092AC058091AC05853108F451C020918D0530918E05809116
S12312E0B4049091B5048217930778F48091A5059091A60582609093A6058093A5058091B4
S1231300A70588608093A70509C08091A5059091A6058D7F9093A6058093A5058091260553
S123132083FF16C080918D0590918E05815D974078F08091A5059091A60584609093A605A4
S12313408093A5058091A70582608093A70509C08091A5059091A6058B7F9093A605809333
S1231360A5058091A90590E09093AB058093AA0584E38093AC0508958091AA059091AB05A2
S1231380892B49F08091AA059091AB0501979093AB058093AA0508959C018091260584FFA5
S12313A01BC022533040C90143E0880F991F4A95E1F7220F331F280F391F2455354F4427FC
S12313C037FD4095542F60E579E784E090E00E943427822F90E008958091260585FD03C0C8
S12313E084E690E0089522533040C901A3E0880F991FAA95E1F7220F331F280F391F24554F
S1231400354F442737FD4095542F60E579E784E090E00E9434272C592695822F90E00895D9
S12314200F931F93CF93DF93CDB7DEB760970FB6F894DEBF0FBECDBFA89582E50E940626B7
S123144083E10E94062680918D0590918E05892F99270E94062680918D0590918E050E94C0
S1231460062680913E0590913F050E94062680913805909139050E940626809128059091DB
S123148029050E94062680913605909137050E94062680913405909135050E940626809151
S12314A03005909131050E94062680919305909194056091180170E00E94EB26CB010E94F0
S12314C00626809192050E940626809191050E94062620911406309115068091E205909131
S12314E0E305F3E096958795FA95E1F78170232F3327822B0E940626809114069091150600
S12315000E9406268091DC050E940626E0919105F0E0EE51FE4F80810E94062680912E05C3
S123152090912F050E9406268091E4059091E505969587950E9406268BB18295817090E0B6
S12315409A8389838BB182958695817090E09C838B8380913606992787FD90959E838D837B
S123156080910706992787FD909598878F838091A70590E09A8789878091A5059091A605CA
S12315809C878B8780913205909133059E878D878091A70590E0988B8F879091B605E92FDE
S12315A0F0E0EE0FFF1F8E010F5F1F4FE00FF11F81819295907F892B0E940626E091B605EC
S12315C0F0E0EE0FFF1FE00FF11F80810E9406268DEA0E9406268091B6058F5F8093B60581
S12315E0883010F01092B60560960FB6F894DEBF0FBECDBFDF91CF911F910F910895CF9277
S1231600DF92EF92FF920F931F93CF93DF93A89588E10FB6F89480936000109260000FBEE2
S12316200E945226882309F49BC50E94E3259093B5058093B4058136910509F486C08236E9
S1231640910508F041C08D34910509F4E4C18E349105E8F48134910509F49FC082349105D7
S123166068F48932910509F4B7C48433910509F45EC58832910509F071C58BC485349105B7
S123168009F4C4C08634910509F068C548C18335910509F4F3C48435910548F4803591056E
S12316A009F439C38235910509F058C5B0C38735910509F4A7C38835910509F438C4853598
S12316C0910509F04BC5EBC38936910509F4D4C28A369105E8F48436910509F441C5853691
S12316E0910548F48236910509F49BC28336910509F034C599C28636910509F4EEC0863617
S1231700910508F4FBC18736910509F027C5DBC28037910509F404C38137910548F48D3644
S1231720910509F437C18F36910509F017C517C48937910509F473C48A37910509F477C2F8
S12317408837910509F00AC572C281E60E94062680EA0E9406261092B5051092B4050EC042
S1231760EE5BFE4F80810E9406268091B4059091B50501969093B5058093B405E091B405F1
S1231780F091B505E03AF10558F38FEF99E50197F1F7000000C08EE9E1C41092B505109259
S12317A0B405C0E0D0E00E945226882341F1C091B405D091B505C03AD10589F40E94E32509
S12317C09093B5058093B4058E3B910519F4C6E1DAEF15C08091B4050E940626FBCF0E94A7
S12317E0E325CE5BDE4F88838091B4059091B50501969093B5058093B405C0E0D0E0219690
S12318004AEFC030D40708F0ABC4CDCFC0E0D0E00E945226882309F459C00E94E3258A3B23
S1231820910509F09DC488E10FB6F89480936000109260000FBE1092B5051092B4053EC003
S1231840885B0E9406268DEF0E9406262091B4053091B5058AEF90E0289FE001299FD00D6E
S1231860389FD00D112407C0DE010E944F27802D0E94062621962091B4053091B5052F5F18
S12318803F4F8AEF90E0AC01249FC001259F900D349F900D112421503040C817D90720F3E3
S12318A0822F885B80950E9406268091B4059091B50501969093B5058093B4058091B405FE
S12318C09091B5058430910508F4BACF21965AEFC030D50708F044C49BCF86E60E940626EA
S12318E080EA0E9406261092B5051092B4050EC0EE51FE4F80810E9406268091B4059091E1
S1231900B50501969093B5058093B405E091B405F091B505E03AF10558F389E91FC4109212
S1231920B5051092B40500E010E00E945226882349F1C091B405D091B505C03AD10591F445
S12319400E94E3259093B5058093B405893B910519F406E11AEF16C0E091AE05F091AF05AA
S1231960099510C00E94E325CE51DE4F88838091B4059091B50501969093B5058093B4050F
S123198000E010E00F5F1F4F8AEF0030180708F0E7C3CBCF8DE60E94062689E00E9406261B
S12319A080911C0190911D010E94062680911C0190911D01892F99270E9406268091220101
S12319C0909123010E9406268091220190912301892F99270E9406268091000190910101FC
S12319E00E9406268091000190910101892F99270E940626809113010E9406268091120183
S1231A000E940626AAE0B0E00E944F27802D0E94062682E9A3C31092B5051092B405C0E01F
S1231A20D0E00E9452268A3008F461C00E94E32590931D0180931C0100911C0110911D0179
S1231A400E94E325982F8827800F911F90931D0180931C010E94E32590932301809322018B
S1231A6000912201109123010E94E325982F8827800F911F90932301809322010E94E32563
S1231A80909301018093000100910001109101010E94E325982F8827800F911F9093010150
S1231AA0809300010E94E325809313010E94E325809312010E94E325AAE0B0E0082E0E94D1
S1231AC05C270E94F81F0E94E325823B910551F40E949E03E091AE05F091AF050995CFE695
S1231AE0DAEF05C0E091AE05F091AF05099521964AEFC030D40708F033C393CF85E60E9445
S1231B00062683E10E9406261092B5051092B4050EC0EE5DFC4F80810E9406268091B405AF
S1231B209091B50501969093B5058093B405E091B405F091B505EA30F10558F3809119019B
S1231B400E94062680911A010E9406268FEF95E30197F1F7000000C0809127010E9406267C
S1231B60809128010E940626809129010E94062680912A010E9406268091140190911501E9
S1231B8066E070E00E94EB26CB010E940626809124010E940626AEE6B1E00E944F27802D70
S1231BA00E9406268AE90E9406268CE60E94062684E10E9406261092B5051092B4050EC01A
S1231BC0E951FA4F80810E9406268091B4059091B50501969093B5058093B405E091B405A0
S1231BE0F091B505EA30F10558F31092B5051092B4050EC0E951FA4F80890E94062680915B
S1231C00B4059091B50501969093B5058093B405E091B405F091B505EA30F10558F383E9C0
S1231C209DC20E9486009CC20E94C10099C20E94100A96C20E94E325C82FD0E00E94E325EE
S1231C40C817D90709F08CC20E94E3258C019093B5058093B4050E94E3250817190709F0B8
S1231C607FC20E94E3258639910509F079C28091B405CE5BDE4F4DC00E9452268530D0F62A
S1231C80FBCF0E94E325C82FD0E00E94E325C817D90709F065C20E94E3258C019093B50588
S1231CA08093B4050E94E3250817190709F058C20E94E3258839910509F052C28091B40580
S1231CC0CE51DE4F26C00E9452268530D0F6FBCF0E94E325C82FD0E00E94E325C817D907B5
S1231CE009F03EC20E94E3258C019093B5058093B4050E94E3250817190709F031C20E9490
S1231D00E3258F3A910509F02BC28091B405CE57DD4F888325C20E9452268530C8F6FBCF0E
S1231D20C0E0D0E00E945226823080F10E94E3250E94E3258F38910509F012C21092B50538
S1231D401092B4051CC0EE57FD4F108180E70E94062682E00E9406268091B4050E94062629
S1231D60812F0E9406268FE80E9406268091B4059091B50501969093B5058093B405E09146
S1231D80B405F091B505E03AF105E8F221965AEFC030D50709F4E4C1C5CF0E94E3258C0128
S1231DA00E94E325D82FCC27C00FD11F0E94E3258C019093B5058093B4050E94E325081713
S1231DC0190709F0CDC10E94E325883A9105A9F4DE010E945727E0708091B4059091B505C5
S1231DE0E82BF92BF093B505E093B405DE010F010E94682712BC11BCB3C1E091AE05F0916B
S1231E00AF0509950E945226853038F6FBCFCC24DD240E9452268330C0F10E94E3258C01FF
S1231E200E94E325EC010E94E3258D3A910509F097C1FC2EEE24E00EF11ED7010E944F2786
S1231E40802D90E0D70111960E944F27002D10E0102F0027080F191F84E50E94062684E05D
S1231E600E940626802F0E9406268E2D0E940626EF2CFF248E2D0E940626012F1127802FAC
S1231E800E9406268BEA0E9406260894C11CD11C80E0C8168AEFD80609F462C1BACFCC2499
S1231EA0DD240E9452268330C0F10E94E3258C010E94E325EC010E94E3258A3A910509F0D4
S1231EC04FC1FC2EEE24E00EF11ED7010E944F27802D90E0D70111960E944F27002D10E0F4
S1231EE0102F0027080F191F85E50E94062684E00E940626802F0E940626012F1127802F2B
S1231F000E9406268E2D0E940626EF2CFF248E2D0E9406268AEA0E9406260894C11CD11CF7
S1231F2040E0C4164AEFD40609F41AC1BACFC0E0D0E00E945226882359F00E94E325873A66
S1231F40910509F00DC1E091AE05F091AF05099521965AEFC030D50709F402C1EACFC0E044
S1231F60D0E00E945226882369F00E94E3258039910509F0F5C00E94FD00E091AE05F091A4
S1231F80AF05099521968AEFC030D80709F4E8C0E8CFC0E0D0E00E9452268823B1F00E9438
S1231FA0E325873D910509F0DBC08091340590913505ADE6B1E0082E0E945C2712BC11BC68
S1231FC0E091AE05F091AF05099521964AEFC030D40709F4C5C0DFCFC0E0D0E00E945226B1
S1231FE08823B1F00E94E325863D910509F0B8C08091340590913505AEE6B1E0082E0E947B
S12320005C2712BC11BCE091AE05F091AF05099521965AEFC030D50709F4A2C0DFCFC0E02E
S1232020D0E00E945226823010F10E94E325892B09F096C00E94E32586389105C1F489E74F
S12320400E94062685E00E9406268FEC0E9406268FE30E94062687E00E94062687ED0E94A7
S1232060062684ED0E94062686E80E94062621968AEFC030D80709F473C0D3CFC0E0D0E094
S12320800E945226823008F44CC00E94E325892B09F047C00E94E3258C3A910509F060C0EB
S12320A083E50E94062688E00E94062680919505909196050E940626809195059091960514
S12320C0892F99270E94062680911206909113060E9406268091120690911306892F9927AA
S12320E00E94062680910B0690910C060E94062680910B0690910C06892F99270E94062650
S123210080914806909149060E9406268091480690914906892F99270E9406268CEA0E94F1
S1232120062621964AEFC030D407D1F0A9CFC0E0D0E00E945226823058F00E94E325892BB9
S123214079F40E94E3258B3C910511F40E94110121965AEFC030D50719F0EBCF0E940626F1
S1232160A895DF91CF911F910F91FF90EF90DF90CF9008950F931F93CF93DF9310921506A0
S1232180109214060E945125259A249A00002D9A2C9A81E080931106399A419A209A219AAF
S12321A0219A209A289A299A299A289A549A559A5C9A5D9A229A239A3A9A2A9A2B98429824
S12321C000000000529853983B983C983A983F980E945825569AAAE5B1E00E944F27802DE2
S12321E080939B050E94A11F0E94F81F0E9441250E9447060E94A2042A9A2B98A7E0B0E030
S12322000E944F27802D12BC11BC85FF9BC080910001909101019F7D9093010180930001F1
S12322200E949E030E94EB030E94C1000E9486000E94FD0086E0AAE0B0E0082E0E945C27C2
S123224089E1ABE0B0E0082E0E945C278EE1ACE0B0E0082E0E945C27AEE0B0E0082E0E94BE
S12322605C2720E030E0F901EE5DFC4F8081D901A25ABE4F082E0E945C272F5F3F4F2A3082
S1232280310589F780912701A9E6B1E0082E0E945C2780912801AAE6B1E0082E0E945C271A
S12322A080912901ABE6B1E0082E0E945C2780912A01ACE6B1E0082E0E945C2720E030E098
S12322C0F901E951FA4F8081D901AE58BE4F082E0E945C272F5F3F4F2A30310589F720E008
S12322E030E0F901E951FA4F8089D901A458BE4F082E0E945C272F5F3F4F2A30310589F7DA
S123230080910A06A1E7B1E0082E0E945C27809114019091150166E070E00E94EB26ADE0F1
S1232320B0E0062E0E945C2784E1ADE6B1E0082E0E945C2781EEAEE6B1E0082E0E945C27DD
S123234012BC11BC0E94E8000E9411010E949A000E946100809100019091010185FD07C0E3
S123236080916F008B7F80936F002D9A2C9A80912601882311F480E801C080E480933801FF
S12323801092270580911401909115018D5A9D4030F08CEA9DE09093150180931401109234
S12323A08A0586B3866086BB78948AEA0E94062680E00E94062685E50E94062686B1829528
S12323C0817080939D0580916E00836080936E002A9A8BB18295869586958370809581702A
S12323E08295880F880F807C9BB19F7B982B9BB92B9AA89580918D0590918E058E37910567
S123240070F180918A05882351F580911406909115069F7E909315068093140680916F0057
S1232420856080936F0080916E00836080936E002A9A81E080938A05809114069091150620
S1232440806290931506809314068091140690911506906290931506809314064AC02091AC
S12324608A05213009F045C080918D0590918E058635910508F03DC080916F008D7F80933E
S12324806F00809170008C7F8093700080916F008B7F80936F0080916E00836080936E00CB
S12324A080911406909115068F7D90931506809314068091140690911506877F909315068F
S12324C080931406289A299A299A289A5C9A5D9A2D9A2C9A2093110610928A058091140621
S12324E0909115069F7D90931506809314061092880580918A058130F9F48091880588235F
S1232500C1F080916F00826080936F008091700083608093700080916E00836080936E0058
S12325208091140690911506886090931506809314062A9A2B9A16C0109288052D9A2C9AC2
S123254081E080931106109288051092B30010929405109293058091400190914101892B8A
S123256009F42A9880912705833009F4D1C0843018F4882371F073C0853009F4FCC18530F7
S123258008F429C1863009F4B0C1873009F078C230C280918B0590918C058536910508F4B1
S12325A072C2E0912705F0E080917800909179008C7F65E070E00E94EB26EE0FFF1FE859A4
S12325C0FA4F7183608380912705C82FD0E0E0912705F0E0EE0FFF1FE85DFA4F80819181CA
S12325E0E0912705F0E0EE0FFF1FE859FA4F20813181880F991F880F991F820F931F880FFA
S1232600991F6AE070E00E94EB26CC0FDD1FC85DDA4F7983688310928C0510928B0581E0DF
S12326208093270581E480937C000E94FF0A0E941E07909317018093160180914001909119
S12326404101892B09F41AC28091400190914101019790934101809340012A9A0FC28091FB
S12326608B0590918C058536910508F40CC210928C0510928B05A89580912705813039F53B
S123268080910801909109012091780030917900820F931F969587959093090180930801BB
S12326A083E00E945E0690932B0580932A0580912A0590912B0590933F0580933E0584E660
S12326C080933A0682E08093270585E41EC080910201909103012091780030917900820F8E
S12326E0931F9695879590930301809302018BE490E090932D0580932C05909339058093B4
S1232700380583E08093270584E480937C00BBC180918B0590918C058536910508F4B3C14F
S1232720E0912705F0E080917800909179009695879596958795EE0FFF1FE859FA4F9183BE
S1232740808380912705C82FD0E0E0912705F0E0EE0FFF1FE85DFA4F80819181E0912705C8
S1232760F0E0EE0FFF1FE859FA4F20813181880F991F880F991F820F931F880F991F6AE013
S123278070E00E94EB26CC0FDD1FC85DDA4F7983688310928C0510928B0584E0809327051E
S12327A08091380180937C000E94FF0AA8958091A4058F5F8093A405843010F01092A405F1
S12327C08091A405982F91709093D7058695817080930D0658C180918B0590918C058159FC
S12327E0914008F450C180912601882329F1E0912705F0E080917800909179009695879523
S123280096958795EE0FFF1FE859FA4F91838083A0912705B0E0E0912705F0E0EE0FFF1F3C
S1232820E859FA4F80819181AA0FBB1FA85DBA4F11969C938E933EC0E0912705F0E08091E3
S1232840780090917900EE0FFF1FE859FA4F9183808380912705C82FD0E0E0912705F0E055
S1232860EE0FFF1FE85DFA4F00811181E0912705F0E0EE0FFF1FE859FA4F808191810E94D1
S123288050079C01220F331F280F391FC801F3E0880F991FFA95E1F7801B910B820F931F62
S12328A06AE070E00E94EB26CC0FDD1FC85DDA4F7983688310928C0510928B0585E08093DE
S12328C0270587E880937C0020919D0586B18295817030E090E02817390709F4CFC0E0913C
S12328E0AE05F091AF050995C9C080918B0590918C058536910508F4C6C0E0912705F0E032
S123290080917800909179009695879596958795EE0FFF1FE859FA4F91838083A0912705E9
S1232920B0E0E0912705F0E0EE0FFF1FE85DFA4F20813181E0912705F0E0EE0FFF1FE859D1
S1232940FA4F80819181820F931F880F991F9695879596958795AA0FBB1FA85DBA4F1196AF
S12329609C938E9310928C0510928B0587E08093270583E47FC080918B0590918C05893C3A
S1232980910508F480C0E0912705F0E08091780090917900EE0FFF1FE859FA4F9183808315
S12329A0A0912705B0E0E0912705F0E0EE0FFF1FE85DFA4F20813181E0912705F0E0EE0F53
S12329C0FF1FE859FA4F80819181820F931F96958795AA0FBB1FA85DBA4F11969C938E9316
S12329E010928C0510928B0586E08093270582E441C080918B0590918C058536910508F4C2
S1232A0042C0E0912705F0E08091780090917900969587959695879590E0EE0FFF1FE859C6
S1232A20FA4F91838083A0912705B0E0E0912705F0E0EE0FFF1FE85DFA4F20813181E0916B
S1232A402705F0E0EE0FFF1FE859FA4F80819181820F931F96958795AA0FBB1FA85DBA4F93
S1232A6011969C938E9310928C0510928B051092270586E480937C000E94FF0AA89503C084
S1232A8081E08093270580918B0590918C05019690938C0580938B0580918D0590918E05FA
S1232AA08B58924008F45BC0809138068F5F809338069091380680913906981708F452C04C
S1232AC0109238068091360590913705E0914E06FF27E7FDF095EA5EF94F208130E082173B
S1232AE0930754F480913606843634F48091360690913706890F17C08091360590913705FE
S1232B00E0914E06FF27E7FDF095EA5EF94F208130E0821793074CF08091360682302CF092
S1232B208091360681508093360680913606E0914E06FF27E7FDF095EA5EF94F208999278A
S1232B4087FD909530E02817390764F4E0914E06FF27E7FDF095EA5EF94F808901C081E0D2
S1232B608093360680918D0590918E058739910508F46DC020913405309135058091240111
S1232B8090E04996281739070CF061C08091DE059091DF0501969093DF058093DE05209108
S1232BA0DE053091DF058091E0059091E1052817390708F440C01092DF051092DE05209155
S1232BC08D0530918E058091D8059091D9050A972817390730F49091DC058091DD05890F4D
S1232BE015C020918D0530918E058091D8059091D90549968217930758F49091DC05809107
S1232C00DB05891728F48091DC0581508093DC059091DC058091DA05891718F48091DA05CF
S1232C2008C09091DC058091DB05981720F48091DB058093DC0580918D0590918E058A58F4
S1232C40924038F48091DA058093DC0502C01092DC058091260582FF1BC080918D059091ED
S1232C608E05805D9740A0F420913405309135058091240190E00596281739074CF481E02F
S1232C8080939F058091140690911506916007C010929F0580911406909115069E7F90936D
S1232CA0150680931406809100019091010192FF27C020918D0530918E0580912E01909123
S1232CC02F0182179307E0F420918D0530918E0580913001909131012817390788F42091E1
S1232CE03405309135058091240190E005962817390734F48091140690911506946005C094
S1232D0080911406909115069B7F90931506809314060E9480080E9456090E94BC07809122
S1232D2000019091010180FF67C080912D0180FF11C08091D605883C28F08091DC058823D1
S1232D40B9F418C09091DC058091D6058695891790F010C080912D0182FF0DC08091D60578
S1232D60883C48F0809114069091150696FF02C05C9A01C05C9880912D0184FF16C0809141
S1232D80D605883C28F08091360618165CF12CC0209136068091D605332727FD309586958D
S1232DA090E0821793070CF11FC080912D0186FF1CC08091D605883CC0F020918D0530918C
S1232DC08E0580913201909133018217930760F4209136053091370580919C0590E0821798
S1232DE0930714F45D9A01C05D988091D605883C28F01092D60502C05C9A5D9A8091D605A0
S1232E008F5F8093D605E5CA1F920F920FB60F9211248F939F9380914F068F5F80934F0626
S1232E2080914F06882309F449C080911406909115069061909315068093140610928A0583
S1232E4080911406909115069F7D909315068093140680916F008B7F80936F0080916F00F4
S1232E608D7F80936F00809170008C7F8093700080916E00836080936E002D9A2C9A81E0E0
S1232E808093110680911406909115068F7D90931506809314068091140690911506877FB9
S1232EA09093150680931406289A299A299A289A5C9A5D9A10928E0510928D0578949F9107
S1232EC08F910F900FBE0F901F90189520914C0630914D0680918400909185002817390796
S1232EE060F580913F068430A1F48091970590919805880F991F90939805809397058091A0
S1232F009705909198058160909398058093970504C0109298051092970581E080933F0609
S1232F208091F3049091F4049093F6048093F5041092F4041092F30405C080913F068F5F07
S1232F4080933F06809184009091850090934D0680934C0608951F920F920FB60F92112475
S1232F608F939F938091F3049091F40401969093F4048093F3049F918F910F900FBE0F90C1
S1232F801F901895282F809114069091150693FD08C0213019F0223021F402C02D980895D6
S1232FA02C9808951F938091CF05882391F18091CF05813061F42D9A1092CF058091F304B8
S1232FC09091F40490935806809357060FC08091CF05823059F42C9A1092CF058091F304EC
S1232FE09091F404909344068093430680910B0690910C06892B49F180914A06882329F182
S123300080910B0690910C0690938B0080938A001CC080914A068823C1F010914A06113041
S123302021F010914A06123031F480914A060E94C2171093CF0580914806909149069093DE
S12330408B0080938A0010924A061F9108951F920F920FB60F9211242F933F934F935F93B0
S12330606F937F938F939F93AF93BF93EF93FF930E94D2172A9A7894FF91EF91BF91AF9141
S12330809F918F917F916F915F914F913F912F910F900FBE0F901F9018951F920F920FB6EE
S12330A00F9211242F938F939F93F89480914006882309F46BC08091A5059091A60597FD4F
S12330C065C02091130120959091E605943001F1953040F4923019F19330A0F4913009F0B5
S12330E049C008C0973169F19336A9F19E3009F041C01BC02093B20084E08093B100289886
S123310083E042C026BD83E085BD299884E03CC02093B2009093B100289882E035C026BD6A
S123312083E085BD299881E02FC081E0809310052093B20084E08093B1002898289887E1D7
S123314023C081E08093110526BD83E085BD299829988EE019C081E0809310052093B200BF
S123316084E08093B10028982898299829989093E6050CC02093B20084E08093B1002898FA
S123318028982998299883E68093E60578949F918F912F910F900FBE0F901F901895CF939D
S12331A0DF93EC0180919A05E7E0F0E0E81BF109EE0FFF1FE85DFA4F80819181209199055D
S12331C0821B282F30E080912B0190E0880F991F880F991FAC01429FC001439F900D529FDD
S12331E0900D112464E670E00E94EB266436710520F083E680934B0602C060934B068091A8
S12332004B066AE00E94DF2680933D0680913D068A301CF089E080933D0680918D05909175
S12332208E05885E934008F0B3C010923B068FEF80934E0680913D06992787FD909564E00A
S1233240880F991F6A95E1F78093910580918D0590918E0564E670E00E94EB26655060934F
S1233260470680918D0590918E05845F914060F410924706E0914706FF27E7FDF095E55C21
S1233280FE4F808190E0A3C0809147068430D9F5E0919105F0E0EE5BFE4F2081E09147065D
S12332A0FF27E7FDF095E55CFE4F6081E0914706FF27E7FDF095E55CFE4F808190E090939D
S12332C0E5058093E405E091E405F091E50580918D0590918E054091470630E0220F331F37
S12332E0261B3109845F91406CE94602A0011124840F951FAC01249FC001259F900D349F7C
S1233300900D11243AC0E0914706FF27E7FDF095E45CFE4F6081E0914706FF27E7FDF095D5
S1233320E55CFE4F4081E0914706FF27E7FDF095E55CFE4F808190E09093E5058093E405E5
S1233340E091E405F091E50580918D0590918E052091470670E0641B7109845F91404CE91D
S1233360240290011124820F931F9C01629FC001639F900D729F900D112464E670E00E94FD
S1233380EB26E60FF71FF093E505E093E405C7C080918D0590918E05875F9242E8F086E965
S12333A080933B068FE080934E0680913D0690914E068295807F890F80939105E0919105B8
S12333C0F0E0EE5BFE4F808190E0880F991F9093E5058093E405A3C080918D0590918E0500
S12333E0885E934062E370E00E94EB2660933B0680913B066AE00E94DF2680934E068091D9
S12334003D0690914E068295807F890F80939105E0919105F0E0EE5BFE4F808190E0880F24
S1233420991F9093E5058093E40580914E0687FD39C080914E068F30ACF5E0919105F0E049
S1233440ED5BFE4F8081E0919105F0E0EE5BFE4F6081E091E405F091E50520913B064091FC
S12334604E06861B880F992787FD909530E06AE04602A0011124241B350BAC01429FC0010D
S1233480439F900D529F900D11246AE070E00E94FF26772767FD70956E0F7F1F7093E50576
S12334A06093E40580913D0687FD39C080913D068930ACF5E0919105F0E0EE5AFE4F808140
S12334C0E0919105F0E0EE5BFE4F6081E091E405F091E50520914B0640913D06861B880F87
S12334E0992787FD909530E06AE04602A0011124241B350BAC01429FC001439F900D529FA9
S1233500900D11246AE070E00E94FF26772767FD70956E0F7F1F7093E5056093E405809178
S1233520140690911506977F90931506809314068091E2059091E305877F9093E30580938B
S1233540E2058091A705882309F458C08091A70588233CF18091A705883088F080913E062C
S123356090E083709070892B09F448C080913E0667E00E94DF26992309F440C012C080914C
S1233580A7058430C0F080913E0690E083709070892B39F080913E0667E00E94DF26992383
S12335A069F580911406909115069860909315068093140623C08091A705823050F080913C
S12335C0E2059091E30588609093E3058093E20515C08091A705882389F08091E405909139
S12335E0E5058739910550F08091E4059091E5058C5890409093E5058093E40580913E0630
S12336008F5F80933E064091B905445645310CF044E12091E4053091E50580911201909117
S12336208905285B3F4F280F311D291B3109842F4C3E0CF48CEE992787FD9095280F391F35
S12336403093B8052093B7058091B7059091B8058D5B92402CF06CEB72E080E090E015C0A8
S12336608091B7059091B80505972CF465E070E080E090E00AC08091B7059091B8059C0168
S1233680B901882777FD8095982F6E537E4F8F4F9F4F20918F05309190052C0F3D1F40E0C1
S12336A050E00E94C02628E037E040E050E00E941227C21BD30BCE01DF91CF910895A0E08D
S12336C0B0E0BC01CD0128E532E040E050E00E94C02628E037E040E050E00E941227DA01AF
S12336E0C90108950F931F93CF93DF938091090590910A05909356068093550680910905DC
S123370090910A05499708F44CC280914F06882349F088EE9DEF90930E0580930D05109242
S12337204F0653C080918D0590918E0540910D0550910E05895B9B40C0F0E0918F05F091FA
S123374090052091090530910A058091F70490E0241B350BAC01429FC001439F900D529F87
S1233760900D112464E170E017C0E0918F05F09190052091090530910A058091F70490E0E1
S1233780241B350BAC01429FC001439F900D529F900D11246EE170E00E94FF26CB018E0F46
S12337A09F1F62E070E00E94FF267093900560938F051092900510928F0580910905909122
S12337C00A0590930E0580930D0580918805893628F4809188058F5F8093880580918D0533
S12337E090918E05C0910D05D0910E05D0931306C0931206209112063091130600910B050F
S123380010910C0540E050E060E070E489E191E00E943427CA01B9012EE130E040E050E042
S12338200E94C02620EC30E0A901049F9001059F300D149F300D11242050324040E050E0CA
S12338400E94122730938E0520938D052091C6053091C7054091C4055091C505C901880F3F
S1233860991F820F931F840F951F96958795969587959093C7058093C6058091C2059091AE
S1233880C3059093C5058093C4058091C0059091C1059093C3058093C2058091BE0590911C
S12338A0BF059093C1058093C0058091BC059091BD059093BF058093BE058091BA0590911C
S12338C0BB059093BD058093BC0580918D0590918E059093BB058093BA0580918D0590919B
S12338E08E058D5D9540B8F08091B9054091BA055091BB052091C6053091C70590E0821BB4
S1233900930B840F951F9695879596958795855B8093B9050FC084E68093B90580918F05D0
S12339209091900564E070E00E94FF267093900560938F0510924F0680918D0590918E0505
S12339408C529140A0F580910B0590910C05039771F580913F06813051F584E090E0909388
S12339600C0580930B0580910B0590910C05806880938100809184009091850096958795BE
S1233980969587959093850080938400D695C795D695C795D0930E05C0930D05809112060B
S12339A09091130696958795969587953AC080918D0590918E058F5E9240B8F180910B0561
S12339C090910C05049789F580913F06813069F583E090E090930C0580930B0580910B05E8
S12339E090910C058068809381008091840090918500880F991F880F991F90938500809381
S1233A008400CC0FDD1FCC0FDD1FD0930E05C0930D058091120690911306880F991F880F4C
S1233A20991F909313068093120680911206909113060E94CF189093490680934806809193
S1233A40E2059091E30583FF3AC0E091D005F091D105CF0183709070892B99F4209112068C
S1233A603091130680911206909113066AE070E00E94EB26261B370B309349062093480622
S1233A8018C020913901809112069091130668E270E00E94EB2630E0629FC001639F900D3E
S1233AA0729F900D11248C599F4F90934906809348063196F093D105E093D00504C01092AB
S1233AC0D1051092D00580918D0590918E058A58924038F080912805909129058E3691057B
S1233AE03CF48CE291E0909353068093520604C01092530610925206809148069091490644
S1233B0020911601309117014091520650915306821B930B841B950B90934206809341065E
S1233B20809141069091420697FF20C08091410690914206209112063091130640914806C7
S1233B4050914906820F931F8417950778F420911206309113068091480690914906821B3C
S1233B60930B44969093420680934106F89480913F06833011F48EE005C080913F0682302F
S1233B8081F487E18093E60580911206909113060E945F1B909389008093880081E080930C
S1233BA040067894DF91CF911F910F9108951F920F920FB60F9211242F933F934F935F939D
S1233BC06F937F938F939F93AF93BF93EF93FF9389B186958695817020919B0590E030E09F
S1233BE082179307C9F00E94721B0E9466178091950590919605880F991F90939605809300
S1233C009505809195059091960581609093960580939505419882C12091840030918500BC
S1233C208091090590910A05969587952817390770F480918D0590918E05815D974038F0D3
S1233C4081E090E0909396058093950567C18091E2059091E30583FF94C08091840090916F
S1233C60850090930A058093090510928500109284008091950590919605880F991F909342
S1233C80960580939505419A20913901809112069091130668E270E00E94EB2630E0629F51
S1233CA0C001639F900D729F900D11248C599F4F909349068093480680918D0590918E05C0
S1233CC08051974208F049C0809114069091150693FD43C0809148069091490690938B00BE
S1233CE080938A00209112063091130680911206909113069695879596958795281B390B08
S1233D0030930C0620930B0680913F06813021F080913F06833031F42C9882E08093CF05B3
S1233D2081E00DC080913F06843021F080913F06823039F42D9881E08093CF0582E080937F
S1233D404A068EEB90E090930F0680930E0680911406909115069F770FC080911206909131
S1233D6013068C509E4F90938B0080938A0080911406909115069068909315068093140648
S1233D80CDC0809184009091850090930A05809309051092850010928400809195059091EB
S1233DA09605880F991F9093960580939505419A80918D0590918E058051974208F0A4C072
S1233DC080914106909142068536910564F11092CF05809141069091420690938B00809380
S1233DE08A0080918A0090918B0090930C0680930B0680913F06813021F080913F06833074
S1233E0011F481E009C080913F06843021F080913F06823029F482E080934A061092CF05F4
S1233E2084E090E06CC080914106909142068B5B9F4F7CF11092CF0584E690E090938B007E
S1233E4080938A0090930C0680930B0680913F06813021F080913F06833011F481E009C018
S1233E6080913F06843021F080913F06823039F482E080934A060E94C2171092CF0588E2CE
S1233E8090E090930F0680930E0684E180930F0545C0809148069091490690938B0080932E
S1233EA08A0020911206309113068091410690914206820F931F90930C0680930B06809163
S1233EC03F06813021F080913F06833029F481E00E94C21781E00CC080913F06843021F08D
S1233EE080913F06823031F482E00E94C21782E08093CF0584E180930F0584EB90E09093DD
S1233F000F0680930E060AC080911206909113068C509E4F90938B0080938A002A9A789450
S1233F20FF91EF91BF91AF919F918F917F916F915F914F913F912F910F900FBE0F901F9063
S1233F4018951092800081EF9FEF909389008093880085EF9FEF90938B0080938A0080E894
S1233F608093810080EC9AED909385008093840083E090E090930C0580930B0580910B052C
S1233F8090910C0580688093810080916F00876080936F0052985398259A249A2D9A2C9AA7
S1233FA081E080931106A2E0B2E00E944F27802D8093F704A1E0B2E00E944F27802D8093A0
S1233FC0F8048091F8048E3039F08091F804873119F087E18093F804809169008460809337
S1233FE0690080916900816080936900E89A089521EB30E0F90110821092B6001092B2000A
S12340001092B300A0E7B0E08C9183608C93209A219A219A209A289A299A299A289AEFE648
S1234020F0E080818D7F80838C918C7F8C9386E0F901808384E6809307060895813099F48D
S1234040289A289A80912C01843021F4299A299A1092110510925C0610925B0610921005D5
S12340601092B1000895823049F4299A299A10925A06109259061092110515BC08951F92FD
S12340800F920FB60F9211242F933F934F935F936F937F938F939F93AF93BF93EF93FF9368
S12340A0F89480911005843019F481E00E941E207894FF91EF91BF91AF919F918F917F913C
S12340C06F915F914F913F912F910F900FBE0F901F9018950F931F93809128059091290534
S12340E00A9714F487E003C080919F0586E08093B1001092B20080918D0590918E05845F7C
S1234100914018F41092470616C080918D0590918E058D56974020F08EE0809347060BC03F
S123412080918D0590918E0564E670E00E94EB26655060934706E0914706F0E0E45DFC4FC8
S123414080818093130180919F05882329F02091F2018091180108C0E0919105F0E0EE510E
S1234160FE4F808120911801829FC00111249093D3058093D20580918D0590918E05825CF2
S1234180914048F5809100019091010182FF19C08091D2059091D30520911901820F911D93
S12341A09093D3058093D2058091140690911506846090931506809314068EE18093D40505
S12341C03FC080911406909115068B7F909315068093140635C080911406909115068B7F9A
S12341E090931506809314068091D405823028F08091D40581508093D405E091D205F0912C
S1234200D30580911901209119014091D405E80FF11D8EE190E0841B910930E0AC01429F67
S1234220C001439F900D529F900D11246EE170E00E94EB26E61BF70BF093D305E093D2057D
S123424080919F05882309F0A3C180914E0687FD3EC080914E068F30D4F5E0919105F0E0F2
S1234260ED51FE4F6081E0919105F0E0EE51FE4F40810091D2051091D30580913B062091C6
S12342804E06E091180170E0641B710990E04AE0240290011124821B930B9C01629FC001D3
S12342A0639F900D729F900D11246AE070E00E94FF26F0E06E9FC0016F9F900D7E9F900D14
S12342C01124800F911F9093D3058093D20580913D0687FD3EC080913D068930D4F5E09164
S12342E09105F0E0EE50FE4F6081E0919105F0E0EE51FE4F40810091D2051091D3058091D2
S12343004B0620913D06E091180170E0641B710990E04AE0240290011124821B930BAC0113
S1234320649FC001659F900D749F900D11246AE070E00E94FF26F0E06E9FC0016F9F900D85
S12343407E9F900D1124800F911F9093D3058093D205809100019091010184FF5CC02091C1
S1234360540530915505809134059091350528173907FCF480913405909135052091540502
S123438030915505821B930B64E070E00E94FF2680919205861710F46093920580919205ED
S12343A08A3018F089E080939205809125018093D5053091D5053430C8F08091D205909140
S12343C0D305E0919205F0E0EE5DFC4F2081820F911D9093D3058093D20531503093D505B0
S12343E08091140690911506806109C0109292051092D50580911406909115068F7E90935C
S123440015068093140680913405909135059093550580935405809100019091010191FFFD
S1234420B4C080919D05882309F0AFC0809109068F5F809309069091090680910A0698170E
S123444008F4A6C0109209068091300590913105E0913D06FF27E7FDF095E951FA4F208141
S123446030E028173907B4F48091300590913105E0913D06FF27E7FDF095E951FA4F2081FD
S1234480821B910962E070E00E94FF266C59609307062BC08091300590913105E0913D0687
S12344A0FF27E7FDF095E951FA4F208130E082179307DCF4809107061816BCF4E0913D0682
S12344C0FF27E7FDF095E951FA4F8081209130053091310590E0821B930B62E070E00E9409
S12344E0FF2684E6861B8093070680911406909115069D7F909315068093140620910706BC
S1234500E0913D06FF27E7FDF095E951FA4F8089332727FD309590E08C599F4F821793070F
S123452054F4E0913D06FF27E7FDF095E951FA4F80898C591EC020910706E0913D06FF2705
S1234540E7FDF095E951FA4F4089332727FD309584E690E0841B910928173907CCF4E0919C
S12345603D06FF27E7FDF095E951FA4F908984E6891B809307068091140690911506926042
S1234580909315068093140603C084E6809307068091D2059091D30520913A0630E062E03B
S12345A070E00E94FF26269FC001279F900D369F900D112464E670E00E94EB26660F771FF8
S12345C07093D3056093D20520913E0530913F0580911B0190E0C296281739070CF046C0C3
S12345E0809100019091010181FF40C080913E0590913F05C397D4F040911A0180911A0113
S123460020913E0530913F0560911B0190E070E06E5C7F4FFC01E29FC001E39F900DF29F49
S1234620900D11240E94EB26461B03C080911A01482F50E08091D2059091D305480F591F4A
S12346405093D3054093D205809120019091210190931F0180931E018091140690911506A0
S12346608260909315068093140611C080911406909115068D7F9093150680931406809129
S12346801C0190911D0190931F0180931E0180912601882371F02091D2053091D3058091CF
S12346A0070624563040992787FD9095280F391F0DC02091D2053091D305809107062C5976
S12346C03F4F992787FD9095281B390B3093D3052093D2058091E2059091E30583FF1CC0D4
S12346E0E091D205F091D30520913A018091D2059091D30564E170E00E94FF2630E0629FDB
S1234700C001639F900D729F900D11248E0F9F1F9093D3058093D2058091000190910101DD
S123472090FF4CC08091280590912905823891050CF044C08091D2059091D3052091270143
S1234740820F911D9093D3058093D205E0912805F0912905609118012091270182E890E027
S12347608E1B9F0B70E0AB01849FB001859F700D949F700D11248FEF90E0FB01E89FB0016A
S1234780E99F700DF89F700D1124882777FD8095982F30E040E050E00E94C02620E43FE1BC
S12347A040E050E00E9412278091D2059091D305820F931F9093D3058093D2052091D20539
S12347C03091D3058091180145EF849FC00111248217930754F480911801849FC001112407
S12347E09093D3058093D2050BC08091D2059091D3051816190624F01092D3051092D205D0
S12348008091D2059091D3059093940580939305809114069091150692FF04C0289A299A0B
S1234820299A289A78941F910F9108951F920F920FB60F9211242F933F934F935F936F939F
S12348407F938F939F93AF93BF93EF93FF93F89420911005223039F0243009F44FC02130C8
S123486009F051C01CC080915B0690915C068F3F9105D1F1C8F180915B0690915C068F5F97
S12348808093B30080915B0690915C068F5F904090935C0680935B062093100534C00E9444
S12348A06A20809193059091940590935C0680935B0680915B0690915C068F3F9105A1F024
S12348C098F080915B0690915C068F5F8093B30080915B0690915C068F5F904090935C066B
S12348E080935B0682E007C080915B0690915C068093B30084E08093100505C081E00E9408
S12349001E20109210057894FF91EF91BF91AF919F918F917F916F915F914F913F912F9132
S12349200F900FBE0F901F9018951F920F920FB60F9211242F933F934F935F936F937F93A3
S12349408F939F93AF93BF93EF93FF93F89420911105223039F0243009F453C0213009F0DB
S123496053C020C08091590690915A068F3F910591F088F08091590690915A068F5F87BDCF
S12349808091590690915A068F5F904090935A068093590633C08091590690915A0687BD47
S12349A084E024C0809193059091940590935A068093590624E025BD16BC8091590690910A
S12349C05A068F3F9105A9F0A0F08091590690915A068F5F87BD8091590690915A068F5FE4
S12349E0904090935A068093590682E0809311050BC08091590690915A0687BD209311059A
S1234A0003C082E00E941E207894FF91EF91BF91AF919F918F917F916F915F914F913F91E1
S1234A202F910F900FBE0F901F9018951F920F920FB60F9211242F933F934F935F936F93F4
S1234A407F938F939F93AF93BF93EF93FF93F89480911105843019F482E00E941E20789482
S1234A60FF91EF91BF91AF919F918F917F916F915F914F913F912F910F900FBE0F901F9018
S1234A801895549A559A5C9A5D9A15BCEEE6F0E080818360808384E085BD16BC82E187BD20
S1234AA0089511B88FEF84B915B887B98AB9089588E98093C1001092C50083E18093C400FD
S1234AC084EA96E0909362068093610690935E0680935D0684E696E09093600680935F060B
S1234AE09093E5068093E406109263061092100608951F920F920FB60F9211248F939F9306
S1234B00EF93FF9380916306882311F1E0916106F091620681918093C600F0936206E0934C
S1234B206106E45EF64030F084EA96E09093620680936106809163068150809363068091B1
S1234B406306882329F48091C1008F7D8093C100FF91EF919F918F910F900FBE0F901F9054
S1234B6018951F920F920FB60F9211242F938F939F93EF93FF938091C600E091E406F091BA
S1234B80E5068083809110068F5F809310068091E4069091E50601969093E5068093E4063C
S1234BA0845A964030F084E696E09093E5068093E406FF91EF919F918F912F910F900FBEA6
S1234BC00F901F90189580911006882319F48FEF9FEF0895F89480911006815080931006A1
S1234BE0E0915F06F09160062191F0936006E0935F06E45AF64030F084E696E09093600684
S1234C0080935F067894822F90E00895982F809163068F33E0F780916306803418F080E0DE
S1234C2090E00895F894809163068F5F80936306E0915D06F0915E06908380915D06909192
S1234C405E06019690935E0680935D06845E964030F084EA96E090935E0680935D0680918E
S1234C60C10080628093C100789481E090E00895CF93DF93EC0104C00E94062681112196A3
S1234C8088818823C9F781E090E0DF91CF91089582E195E00E94382608958AE195E00E9467
S1234CA0382608958091100690E00895CF92DF92EF92FF920F931F93CF93DF93CDB7DEB79C
S1234CC029970FB6F894DEBF0FBECDBF8C01F62EE42EDE011196EDE1F5E089E001900D9244
S1234CE08150E1F749E06E010894C11CD11CFF2081F089E090E0841B91092F2D30E0821762
S1234D00930738F04150F601E40FF11D8CE28083FF244150F601E40FF11DC8016AE070E0C4
S1234D200E94EB26805D8083C8016AE070E00E94EB268B01672B11F4FF2019F085E08F1572
S1234D40B0F619E01E197E010894E11CF11C07C0F701E10FF11D80810E9406261F5F193001
S1234D60B8F329960FB6F894DEBF0FBECDBFDF91CF911F910F91FF90EF90DF90CF900895E5
S1234D80629FD001739FF001829FE00DF11D649FE00DF11D929FF00D839FF00D749FF00DC3
S1234DA0659FF00D9927729FB00DE11DF91F639FB00DE11DF91FBD01CF0111240895991B61
S1234DC079E004C0991F961708F0961B881F7A95C9F780950895AA1BBB1B51E107C0AA1F1F
S1234DE0BB1FA617B70710F0A61BB70B881F991F5A95A9F780959095BC01CD01089597FBF5
S1234E00092E07260AD077FD04D0E5DF06D000201AF4709561957F4F0895F6F790958195B2
S1234E209F4F0895A1E21A2EAA1BBB1BFD010DC0AA1FBB1FEE1FFF1FA217B307E407F5078A
S1234E4020F0A21BB30BE40BF50B661F771F881F991F1A9469F760957095809590959B017C
S1234E60AC01BD01CF01089597FB092E05260ED057FD04D0D7DF0AD0001C38F450954095CA
S1234E80309521953F4F4F4F5F4F0895F6F790958095709561957F4F8F4F9F4F0895F99931
S1234EA0FECFB2BDA1BDF89A119600B40895F7DFE02DF5DFF02D0895F999FECFB2BDA1BD2D
S1234EC000BC11960FB6F894FA9AF99A0FBE0895F3DF012CF1DF11240895FFCF2F000100EA
S1234EE002000300040005000600070008003228E803900106141E3C581B581B8813641943
S1234F00121E01010203040A0411C4098813C4096400DCE64003020A143246965000548142
S1234F209596B7AFC3C8BEBEB9B0AFAFADAC4984C0CBD2D6D7D0C7C2BBB8B3AEAAA9458A8F
S1234F40A2A9AAB7C0BABEBBB6B8B2B3B4B93281868DA4A58B8C8F9EA6A2A6A5A6C034529C
S1234F605D5B596F788285858281FF859FB034444E4B4A54615769727272737D9095272C45
S1234F801B252B334B5155616A6D6C7D828B1D211A242A32454C4F5E6169717E8186343214
S1234FA03232323232323232327F323232323232323232323232323232323232323213179A
S1234FC018191B1C1D1F21232527282C2E311418191A1C2124272B3035393C3E4143161909
S1234FE01D232A31353B3F42484E565A5E651B1D363E525863666C6E777D84898D932226B6
S1235000434B6172818A9097A8ACAFB1B6B9292E484E6B7C939BA2AFB9BFCBD2D2D229346D
S12350204B536E7F9CA8B1BCC5D0D2D2D2D2283F4E587187A4B2BAC2D2D2D2D2D2D2374613
S1235040545E7691B1BEC4D2D2D2D2D2D2D239485660869FBAD2D2D2D2D2D2D2D2D200002A
S123506000000000000000000000000000000000000000000000000000000000000000002C
S1235080000000000000000000000000000000000000000000000000000000000000010209
S12350A0030405060708090A0B0C0D0E0F100102030405060708090A0B0C0D0E0F100102DC
S12350C0030405060708090A0B0C0D0E0F1014161718191A1B1C1D1E1F2021222324191A4D
S12350E01B1C1D1E1F2021222324252627271E1F2022232425262728292A2B2C2D2E000271
S123510004060708090A0C0E28262422201E1E1E1E1E1E1E1E1E1E1EF0FF80BBE08804654C
S1235120484BA438022BF0207019CC13860F440CC209D0074C061B052A046A03D102560298
S1235140F201A1015F012801FB00D600B7009D0087007500660059004D0044003C0034004C
S12351602E0029002500F0FF80BBE0880465484BA438022BF0207019CC13860F440CC209F0
S1235180D0074C061B052A046A03D1025602F201A1015F012801FB00D600B7009D00870032
S12351A07500660059004D0044003C0034002E0029002500F0FF80BBE0880465484BA438D0
S12351C0022BF0207019CC13860F440CC209D0074C061B052A046A03D1025602F201A101D2
S12351E05F012801FB00D600B7009D0087007500660059004D0044003C0034002E002900EA
S12352002500F0FF80BBE0880465484BA438022BF0207019CC13860F440CC209D0074C067D
S12352201B052A046A03D1025602F201A1015F012801FB00D600B7009D00870075006600DF
S123524059004D0044003C0034002E00290025000000F5047E05AE066C08C00AB30D630FD4
S12352608B10D7118813000000000A000F001E003C007800FA007201E001800280020000CF
S123528008000A000C000E00C80A4A067E048403AC0D641A002000270032003E0066008ED1
S12352A000B202EB02240337034B03560361037003E800D600C200B0009D008A0078007823
S12352C0006500520040002D001900070000000100010001175A5A5A5050505050505050DE
S12352E050505050506400030000FA3204041B5B481B5B324A000D0A0020202020202020D8
S1055300202067
S503029961
